:020000040800F2
:100000000000082411110008990F00089F0F000834
:10001000A50F0008AB0F0008B10F0008000000009A
:10002000000000000000000000000000B70F000802
:10003000C50F000800000000D30F0008E10F000802
:1000400061110008611100086111000861110008C8
:1000500061110008611100086111000861110008B8
:1000600061110008611100086111000861110008A8
:100070006111000861110008611100086111000898
:10008000611100086111000861110008E503000812
:10009000ED0F0008F90300080D04000861110008C5
:1000A0006111000861110008611100086111000868
:1000B0006111000861110008611100086111000858
:1000C0006111000861110008611100086111000848
:1000D0006111000861110008611100086111000838
:1000E00061110008611100080000000061110008A2
:1000F0006111000861110008611100086111000818
:100100006111000861110008611100086111000807
:1001100061110008611100086111000861110008F7
:1001200061110008611100086111000861110008E7
:100130006111000861110008611100082104000824
:1001400000000000000000000000000000000000AF
:1001500061110008611100086111000861110008B7
:1001600061110008611100086111000861110008A7
:100170006111000861110008611100080000000011
:100180006111000861110008611100086111000887
:100190006111000861110008611100086111000877
:1001A0006111000861110008611100086111000867
:1001B0006111000861110008611100086111000857
:1001C0006111000861110008611100086111000847
:1001D0006111000861110008611100086111000837
:1001E0006111000861110008611100086111000827
:1001F0006111000861110008611100086111000817
:100200006111000861110008611100086111000806
:1002100061110008611100086111000861110008F6
:100220006111000861110008611100080000000060
:100230006111000861110008000000006111000850
:1002400061110008611100086111000861110008C6
:1002500061110008611100086111000861110008B6
:1002600061110008611100086111000861110008A6
:100270006111000861110008611100080000000010
:100280006111000861110008611100080000000000
:080290000000000061110008EC
:1002980010B5054C237833B9044B13B10448AFF3B8
:1002A80000800123237010BD10000024000000000E
:1002B800E856000808B5034B1BB103490348AFF3E0
:1002C800008008BD0000000014000024E856000863
:1002D80080B500AF00F05AFC00BF80BD80B500AF0C
:1002E800024800F03FFD00BF80BD00BFBC020024F3
:1002F80080B582B000AF786039607B68194A934254
:100308002BD1194B194A4021786801F08FFB03461D
:10031800002B22D100220221786801F0F5FC134B52
:100328001B68B3F5887F0AD1104B5B68002B06D198
:100338000D4B1B78552B02D10D4B01221A700B4B1C
:100348001B6840F22222934207D1084B5B68002BBE
:1003580003D10021042000F03FFA00BF0837BD4652
:1003680080BD00BFBC020024F4000024CC0000249F
:100378005C03002480B582B000AF78600B46FB7048
:10038800FB78082B22D8134B40F2FF121A60114B4E
:1003980000225A600F4B00229A60FB781B040D4A1A
:1003A800D3600C4B00221A610A4B00225A61094B98
:1003B80000229A61074B0022DA61064B00221A627A
:1003C8007A680449044801F0D6FA00E000BF08370B
:1003D800BD4680BD34010024BC02002480B500AFB6
:1003E800024801F00BFD00BF80BD00BF2C000024B7
:1003F80080B500AF024801F001FD00BF80BD00BF1D
:100408002C00002480B500AF024801F0F7FC00BFC3
:1004180080BD00BFBC02002480B500AF034801F0D6
:10042800EDFC034801F0EAFC00BF80BD2C0000246D
:10043800BC02002480B485B000AF78600023FB6064
:100448007B68504A934203D87B68B3F1006F07D2A8
:100458007B684D4A934206D87B68B3F1016F02D39B
:100468000023FB6086E07B68484A934203D87B6898
:10047800444A934207D87B68454A934206D87B682A
:10048800414A934202D90123FB6073E07B68414AE9
:10049800934203D87B683D4A934207D87B683E4A1B
:1004A800934206D87B683A4A934202D90223FB60FA
:1004B80060E07B68394A934203D87B68354A9342A7
:1004C80007D87B68364A934206D87B68324A9342FB
:1004D80002D90323FB604DE07B68324A934203D87C
:1004E8007B682E4A934207D87B682F4A934206D8E6
:1004F8007B682B4A934202D90423FB603AE07B686D
:100508002A4A934203D87B68264A934207D87B68D5
:10051800274A934206D87B68234A934202D9052387
:10052800FB6027E07B68234A934203D87B681F4A15
:10053800934207D87B68204A934206D87B681C4AB6
:10054800934202D90623FB6014E07B68B3F1016F84
:1005580003D27B68174A934207D87B68174A9342AD
:1005680006D87B68144A934202D90723FB6001E04E
:100578000723FB60FB6818461437BD465DF8047B0B
:10058800704700BFFFFF0108FFFF1108FFFF0308C6
:10059800FFFF1308FFFF0508FFFF1508FFFF070807
:1005A800FFFF1708FFFF0908FFFF1908FFFF0B08E7
:1005B800FFFF1B08FFFF0D08FFFF1D08FEFF1F08B8
:1005C80080B487B000AFF860B9607A60FA687B6879
:1005D8001344B3F1026F01D903232BE07B68002B8E
:1005E80001D1002326E00123FB7400237B6117E07F
:1005F800FB681B78BB74BB681B78BA7C9A4206D030
:10060800BB7CFF2B01D0022314E00023FB74FB68A2
:100618000133FB60BB680133BB607B6901337B61DD
:100628007A697B689A42E3D3FB7C012B01D10023D2
:1006380000E0012318461C37BD465DF8047B70476F
:1006480080B58CB000AF78600023FB620023BB62EA
:100658000023FB6002F072F97868FFF7EBFEF8629E
:100668000123BB6200233B6120233B627B68B3F11B
:10067800016F02D302237B6101E001237B61FB6AE6
:10068800BB61BB6AFB6107F10C0207F1100311465D
:10069800184602F053FA034687F8273002F088F923
:1006A80097F8273018463037BD4680BD80B592B0E0
:1006B80000AFF860B9607A60FA687B681344B3F1F8
:1006C800026F01D9012382E07B68002B01D100234E
:1006D8007DE07A68B968F868FFF772FF034687F823
:1006E800433097F84330002B01D100236FE00123FA
:1006F800FB63FB6B83F3108800BF02F01FF9002334
:100708007B6419E007F110032022B968184604F049
:10071800D1FFBB682033BB6007F110031A46F968A4
:10072800012002F079F80346002B44D1FB682033FE
:10073800FB607B6C01337B647B685B097A6C9A4253
:10074800E0D37B6803F01F03002B2AD04FF0000290
:100758004FF00003C7E904234FF000024FF00003F5
:10076800C7E906234FF000024FF00003C7E908234A
:100778004FF000024FF00003C7E90A237B6803F03B
:100788001F0207F11003B968184604F093FF07F138
:1007980010031A46F968012002F03EF80346002BC0
:1007A8000BD102F005F90023BB63BB6B83F3108800
:1007B80000BF00230BE000BF00E000BF02F0F8F824
:1007C80000237B637B6B83F3108800BF01231846EB
:1007D8004837BD4680BD000080B483B000AF0346F3
:1007E8003960FB80134B93F841311946114AFB8855
:1007F80022F831300F4B93F841310E4ADB00134495
:100808003A685A600B4B93F841310133DAB2094B1D
:1008180083F84121074B93F84131272B03D9054B26
:10082800002283F8412100BF0C37BD465DF8047BE8
:10083800704700BF5801002480B485B000AF7860CD
:10084800184B93F84021174B93F841319A4201D144
:10085800002320E0134B93F84031DB00114A134486
:10086800FB60104B93F840310133DAB20D4B83F83B
:1008780040210C4B93F84031272B03D9094B002218
:1008880083F84021FB681A887B681A80FB685A68DD
:100898007B685A60012318461437BD465DF8047B0F
:1008A800704700BF5801002480B588B000AF00230E
:1008B8003B610023FB600023BB6100F061F93B460C
:1008C8001846FFF7B9FF0346002B00F0DD803B8890
:1008D800042BF4D16E4B1B78FB72FB7A242B7AD154
:1008E8006B4B5B781A466B4B1A60694B9B781A46C0
:1008F800674BDB781B021A44654B1B791B041A44AF
:10090800634B5B791B0613441A46634B1A60624BB0
:100918001A68624B1B689A424FD1614B1B68002BC7
:100928004BD15B4B9B791A46594BDB791B0213441D
:100938001A465C4B1A605C4B00221A600023FB7558
:100948000CE0FB7D0833524AD35C1A46564B1B68B1
:100958001344554A1360FB7D0133FB75FA7D4D4BFB
:100968001B689A42EDD34F4B1A684F4B1B689A424B
:100978001CD14B4B1B68002B18D1BA694B4B134445
:10098800444A12684A491846FFF790FE0346BB726C
:10099800404B1B68BA691344BB61BB7A002B0BD070
:1009A8003F4B1B6801333E4A136005E03C4B1B6814
:1009B80001333B4A136009E008E0394B1B680133F7
:1009C800374A136004213248FFF7D4FC334B1B68C5
:1009D8000133324A1360FB7A232B0CD1304B1B684E
:1009E800002B08D103212A48FFF7C4FC0A2000F095
:1009F80047FC00F063F8FB7A2A2B47D1244B5B783D
:100A08001A46234B9B781B021A44214BDB781B04A4
:100A18001A441F4B1B791B0613441A46254B1A60B0
:100A2800244B1B68244A1360224B1B685B0C3B61F8
:100A3800204B1B68C3F31003FB60194B00221A609C
:100A4800164B00221A60184B00221A600023BB6163
:100A58000023FB6109E0FB6903F201435B041846CC
:100A6800FFF7EEFDFB690133FB61FA693B699A42C6
:100A7800F1D3FB68002B09D0FB6903F201435B0447
:100A88001846FFF7DDFD01E000BF18E700BF16E7D5
:100A9800F4000024A0020024AC020024B0020024C8
:100AA800A8020024B4020024B802002400000208AE
:100AB800FC000024A40200249C02002480B586B017
:100AC80000AF00237B610123FB60FB6883F3108880
:100AD80000BFFFF703FC254BD3F8E030234A23F08F
:100AE8008003C2F8E030214BD3F8E0301F4A23F0EE
:100AF8000203C2F8E03002F087FC1D4B00221A60A6
:100B08001B4B00225A601A4B00229A6000237B611B
:100B180010E0184A7B6920334FF0FF3142F8231068
:100B2800144A7B6960334FF0FF3142F823107B6928
:100B380001337B617B69072BEBD900233B603B6862
:100B480083F3108800BF0C4B1B683B610B4B1B6881
:100B58007B607B6883F3088800BF0023BB60BB68A9
:100B680083F3148800BF3B699847FEE700440258A6
:100B780010E000E000E100E00400020800000208C4
:100B880080B500AFFFF7A4FB00BF80BD80B500AF04
:100B98003B4B3C4A1A603A4B4FF480729A60384B90
:100BA8000022DA60364B00221A74354B00225A7440
:100BB800334B00229A74324B0A225A61304B01227D
:100BC8009A612F4B0522DA612D4B02221A622C4BB7
:100BD8000A225A622A4B01229A62294B0522DA62BA
:100BE800274B02221A63264B00225A63244B002209
:100BF8009A63234B0022DA63214B20221A64204B8C
:100C080012225A641E4B00229A641D4B1222DA6487
:100C18001B4B00221A651A4B12225A65184B0022E8
:100C28009A65174B0022DA65154B20221A66144B79
:100C380000225A66124B12229A66114800F092FC62
:100C48000346002B01D000F083F9002201210C4853
:100C580001F05AF80346002B01D000F079F9002280
:100C68004FF00071064801F04FF80346002B01D001
:100C780000F06EF9024800F053FE00BF80BD00BFCF
:100C8800BC02002400A4004080B5B8B000AF786072
:100C980007F1CC0300221A605A609A60DA601A6180
:100CA80007F11003BC220021184604F011FD7B68EF
:100CB8001B68294A93424AD14FF400433B614FF0E5
:100CC8008053FB6707F11003184603F025FC034621
:100CD800002B01D000F03CF9204BD3F8EC301F4A30
:100CE80043F48073C2F8EC301C4BD3F8EC3003F4B7
:100CF8008073FB60FB68194BD3F8E030174A43F068
:100D08000203C2F8E030154BD3F8E03003F00203D9
:100D1800BB60BB686023C7F8CC300223C7F8D0306B
:100D28000023C7F8D4300023C7F8D8300923C7F800
:100D3800DC3007F1CC031946094802F071F80022AB
:100D48000021142000F0CBFB142000F0E2FB00BFD0
:100D5800E037BD4680BD00BF00A4004000440258F3
:100D68000004025880B582B000AF78607B681B68C9
:100D78000A4A93420ED10A4BD3F8EC30084A23F4BE
:100D88008073C2F8EC306021064802F0F9F91420AB
:100D980000F0CDFB00BF0837BD4680BD00A4004071
:100DA800004402580004025880B483B000AF124BCC
:100DB800D3F8E030104A43F08003C2F8E0300E4B1D
:100DC800D3F8E03003F080037B607B680A4BD3F8EC
:100DD800E030094A43F00203C2F8E030064BD3F88A
:100DE800E03003F002033B603B6800BF0C37BD46B0
:100DF8005DF8047B704700BF0044025880B500AF1F
:100E080000F0ACF900F02AF8FFF7CEFFFFF7BEFEBE
:100E18000A2000F035FA01210E48FFF7ABFA6420EA
:100E280000F02EFA0C4B1B78002B09D00221094840
:100E3800FFF7A0FA0A2000F023FAFFF735FD08E0D3
:100E480003210448FFF796FA0A2000F019FAFFF781
:100E580035FEFEE7F40000245C03002480B59CB056
:100E680000AF07F124034C220021184604F030FC9F
:100E78003B1D20220021184604F02AFC022002F023
:100E880089FA00233B60304BDB6A2F4A23F00103C9
:100E9800D3622D4BDB6A03F001033B602B4B9B694C
:100EA8002A4A43F440439361284B9B6903F4404327
:100EB8003B603B6800BF254B9B6903F40053B3F5C7
:100EC800005FF8D101237B624FF48033BB620223B9
:100ED800BB640223FB6402233B6540237B6502233A
:100EE800BB651423FB6502233B660C237B6600234A
:100EF800BB660023FB6607F12403184602F0AEFB2D
:100F08000346002B01D000F023F83F237B60032326
:100F1800BB600023FB6008233B6140237B614023C7
:100F2800BB614FF48063FB6140233B623B1D0221A0
:100F3800184602F0C1FF0346002B01D000F008F864
:100F480000BF7037BD4680BD0004005800480258F5
:100F580080B400AF72B600BFFEE7000080B483B073
:100F680000AF0A4BD3F8F430084A43F00203C2F842
:100F7800F430064BD3F8F43003F002037B607B684F
:100F880000BF0C37BD465DF8047B7047004402582B
:100F980080B400AFFEE780B400AFFEE780B400AFD6
:100FA800FEE780B400AFFEE780B400AFFEE780B490
:100FB80000AF00BFBD465DF8047B704780B400AF4A
:100FC80000BFBD465DF8047B704780B400AF00BF2A
:100FD800BD465DF8047B704780B500AF00F030F97E
:100FE80000BF80BD80B500AF024800F007FF00BF1A
:100FF80080BD00BFBC02002480B400AF374BD3F8DB
:101008008830364A43F47003C2F88830344B1B6882
:1010180003F00F03062B07D8314B1B6823F00F038F
:101028002F4A43F0070313602E4B1B682D4A43F0E9
:10103800010313602B4B00221A612A4B1A682949B5
:10104800294B13400B60264B1B6803F00803002B49
:1010580007D0234B1B6823F00F03214A43F00703F3
:101068001360204B00229A611E4B0022DA611D4B4F
:1010780000221A621B4B1D4A9A621A4B1C4ADA62FA
:10108800184B1C4A1A63174B00225A63154B194A0E
:101098009A63144B0022DA63124B164A1A64114BF6
:1010A80000225A640F4B1B680E4A23F480231360F6
:1010B8000C4B00221A66104B1A68104B1340B3F100
:1010C800005F02D20E4B01221A600E4B43F2D2028D
:1010D8001A6000BFBD465DF8047B704700ED00E074
:1010E80000200052004402587FEDF6EA0002020296
:1010F8000000FF01800201010010005C0000FFFFFA
:101108000881005100400052DFF834D0FFF774FF27
:101118000C480D490D4A002302E0D458C45004334A
:10112800C4188C42F9D30A4A0A4C002301E0136020
:101138000432A242FBD304F099FAFFF75FFE70472E
:101148000000082400000024100000247457000840
:101158001000002480030024FEE7000080B582B060
:1011680000AF032000F0B0F903F05CF80246154B1D
:101178009B691B0A03F00F031349CB5C03F01F03A1
:1011880022FA03F37B600F4B9B6903F00F030E4AAF
:10119800D35C03F01F037A6822FA03F30B4A136047
:1011A8000B4A7B6813600F2000F014F80346002BED
:1011B80001D0012302E0FFF7D1FE002318460837CB
:1011C800BD4680BD004402584C5700080400002466
:1011D8000000002480B582B000AF7860154B1B7802
:1011E800002B01D1012321E0134B1A68114B1B7806
:1011F80019464FF47A73B3FBF1F3B2FBF3F31846D5
:1012080000F0A3F90346002B01D001230EE07B6810
:101218000F2B0AD8002279684FF0FF3000F05FF9F1
:10122800064A7B681360002300E00123184608374C
:10123800BD4680BD0C0000240000002408000024E6
:1012480080B400AF064B1B781A46064B1B68134444
:10125800044A136000BFBD465DF8047B704700BFB9
:101268000C0000246003002480B400AF034B1B680B
:101278001846BD465DF8047B704700BF6003002434
:1012880080B584B000AF7860FFF7EEFFB8607B6888
:10129800FB60FB68B3F1FF3F05D00A4B1B781A4689
:1012A800FB681344FB6000BFFFF7DEFF0246BB6824
:1012B800D31AFA689A42F7D800BF00BF1037BD4664
:1012C80080BD00BF0C00002480B400AF034B1B6836
:1012D8001B0C1846BD465DF8047B70470010005C87
:1012E80080B485B000AF78607B6803F00703FB60CB
:1012F8000B4BDB68BB60BA684FF6FF031340BB605B
:10130800FB681A02BB681A43064B1343BB60044AC6
:10131800BB68D36000BF1437BD465DF8047B7047D7
:1013280000ED00E00000FA0580B400AF044BDB6874
:101338001B0A03F007031846BD465DF8047B704797
:1013480000ED00E080B483B000AF0346FB80B7F93E
:101358000630002B0BDBFB8803F01F020749B7F9A7
:1013680006305B09012000FA02F241F8232000BF91
:101378000C37BD465DF8047B704700BF00E100E014
:1013880080B483B000AF0346FB80B7F90630002B6A
:1013980012DBFB8803F01F020A49B7F906305B0924
:1013A800012000FA02F2203341F82320BFF34F8FC7
:1013B80000BFBFF36F8F00BF00BF0C37BD465DF89D
:1013C800047B704700E100E080B483B000AF0346BF
:1013D8003960FB80B7F90630002B0ADB3B68DAB2CC
:1013E8000C49B7F906301201D2B20B4483F8002336
:1013F8000AE03B68DAB20849FB8803F00F03043BB4
:101408001201D2B20B441A7600BF0C37BD465DF804
:10141800047B704700E100E000ED00E080B489B093
:1014280000AFF860B9607A60FB6803F00703FB61FE
:10143800FB69C3F10703042B28BF0423BB61FB69C5
:101448000433062B02D9FB69033B00E000237B61D0
:101458004FF0FF32BB6902FA03F3DA43BB681A4064
:101468007B699A404FF0FF317B6901FA03F3D94356
:101478007B680B40134318462437BD465DF8047B50
:101488007047000080B582B000AF78607B68013B90
:10149800B3F1807F01D301230FE00A4A7B68013B47
:1014A80053600F214FF0FF30FFF78EFF054B0022EE
:1014B8009A60044B07221A60002318460837BD4675
:1014C80080BD00BF10E000E080B582B000AF78605A
:1014D8007868FFF705FF00BF0837BD4680BD80B5B7
:1014E80086B000AF0346B9607A60FB81FFF71CFF46
:1014F80078617A68B9687869FFF790FF0246B7F9AA
:101508000E3011461846FFF75FFF00BF1837BD467B
:1015180080BD80B582B000AF0346FB80B7F90630C6
:101528001846FFF70FFF00BF0837BD4680BD80B5DE
:1015380082B000AF0346FB80B7F906301846FFF7C4
:101548001FFF00BF0837BD4680BD80B582B000AF21
:1015580078607868FFF796FF034618460837BD4657
:1015680080BD000080B598B000AF7860844A07F16C
:101578000C0311464C22184604F09CF87B68002B9B
:1015880001D10123C6E17B681B687E4A934206D1DC
:101598007B681B6803F580731A467B685A607B6812
:1015A80093F89830DBB2002B06D17B68002283F8D1
:1015B80099207868FFF768FB7B681B689A697B68E5
:1015C8001B6822F010029A61FFF74EFEF86514E0DE
:1015D800FFF74AFE0246FB6DD31A0A2B0DD97B682A
:1015E800D3F89C3043F001027B68C3F89C207B68E9
:1015F800032283F8982001238CE17B681B689B6990
:1016080003F00803082BE3D07B681B689A697B68A2
:101618001B6842F001029A61FFF726FEF86514E0A4
:10162800FFF722FE0246FB6DD31A0A2B0DD97B6801
:10163800D3F89C3043F001027B68C3F89C207B6898
:10164800032283F89820012364E17B681B689B6967
:1016580003F00103002BE3D07B681B689A697B6861
:101668001B6842F002029A617B681B7C012B08D13F
:101678007B681B689A697B681B6822F040029A6144
:1016880007E07B681B689A697B681B6842F0400228
:101698009A617B685B7C012B08D17B681B689A691F
:1016A8007B681B6842F480429A6107E07B681B688C
:1016B8009A697B681B6822F480429A617B689B7CEC
:1016C800012B08D17B681B689A697B681B6822F428
:1016D80080529A6107E07B681B689A697B681B687F
:1016E80042F480529A617B681B689B6923F44071BD
:1016F8007B689A687B681B680A439A617B681B68E9
:101708009A697B681B6822F0A4029A617B681B684F
:101718001A697B681B6822F010021A617B68DB6813
:10172800012B08D17B681B689A697B681B6842F0AB
:1017380004029A6130E07B68DB68002B2CD07B6860
:10174800DB68022B20D07B681B689A697B681B6862
:1017580042F080029A617B681B681A697B681B6883
:1017680042F010021A617B68DB68032B14D17B6896
:101778001B689A697B681B6842F020029A610BE03B
:101788000057000800A000407B681B689A697B68C6
:101798001B6842F020029A617B689B69013B5A06EC
:1017A8007B68DB69013B1B021A437B681B6A013BB0
:1017B80042EA03017B685B69013B1A047B681B688A
:1017C8000A43DA617B689B68B3F5407F15D17B6873
:1017D8009B6A5A1E7B68DB6A013B1B021A437B68C3
:1017E8001B6B013B1B0142EA03017B685B6A013BFF
:1017F8001A047B681B680A43DA607B681B6E002B3F
:101808000AD07B681B68D3F8C0107B685A6E7B6867
:101818001B680A43C3F8C0207B68DA6D7B681B6EBF
:101828001344002B11D07B681B68D3F8C83023F011
:1018380007017B689B6E9B0060333B4453F8542C34
:101848007B681B680A43C3F8C8207B681B6C002BA5
:1018580011D07B681B68D3F8BC3023F007017B6884
:101868005B6C9B0060333B4453F8542C7B681B68CB
:101878000A43C3F8BC207B689B6C002B12D07B68A2
:101888001B68D3F8BC3023F070017B68DB6C9B00CD
:1018980060333B4453F8543C1A017B681B680A4385
:1018A800C3F8BC207B681B6D002B12D07B681B68BB
:1018B800D3F8BC3023F4E0617B685B6D9B00603338
:1018C8003B4453F8543C1A027B681B680A43C3F82C
:1018D800BC207B681B68114A934207D17B685B6810
:1018E8009A687B685B6822F003029A607B68002232
:1018F800C3F894207B680022C3F89C207B680122EF
:1019080083F89820786800F083FD034687F85B30F9
:1019180097F85B3018466037BD4680BD00A0004090
:1019280080B483B000AF78607B6893F89830DBB2FE
:10193800012B11D17B68022283F898207B681B68F1
:101948009A697B681B6822F001029A617B68002211
:10195800C3F89C20002308E07B68D3F89C3043F050
:1019680004027B68C3F89C20012318460C37BD4647
:101978005DF8047B704780B586B000AFF860B96049
:101988007A60FB6893F89830DBB2022B41D1FB6890
:101998001B68D3F8C03003F07C53002B09D1FB68D7
:1019A800D3F89C3043F02002FB68C3F89C20012345
:1019B80038E0FB681B68D3F8C43003F40013002B2D
:1019C80009D0FB68D3F89C3043F40072FB68C3F875
:1019D8009C20012326E0FB681B68D3F8C4301B0C4D
:1019E80003F01F037B617B697A68B968F86800F0C7
:1019F80095FEFB681B6801217A6901FA02F2C3F8B7
:101A0800D02001227B699A40FB68C3F89420002308
:101A180008E0FB68D3F89C3043F00802FB68C3F881
:101A28009C20012318461837BD4680BD80B48BB072
:101A380000AFF860B9607A603B600023FB61FB6827
:101A480093F89830FB76FB7E022B40F04B81BB6805
:101A5800402B4DD1FB681B68D3F8A03003F4FE037C
:101A6800002B09D1FB68D3F89C3043F02002FB68B7
:101A7800C3F89C2001233EE1FB681B68D3F8A4301F
:101A880003F07F03002B09D1FB68D3F89C3043F4A3
:101A98008072FB68C3F89C2001232CE1FB681B685B
:101AA800D3F8A4301B0E03F00103012B0BD1FB6804
:101AB8001B68D3F8A030DB0F03F00103B3F1004F2C
:101AC80001D10123FB61FB681B68D3F8A4301B0A12
:101AD80003F03F03FA691344FB61FB685A6FFB6824
:101AE8005B6CF96901FB03F39B0013447B6269E0BB
:101AF800BB68412B4DD1FB681B68D3F8B03003F4A9
:101B0800FE03002B09D1FB68D3F89C3043F0200278
:101B1800FB68C3F89C200123EDE0FB681B68D3F841
:101B2800B43003F07F03002B09D1FB68D3F89C3055
:101B380043F48072FB68C3F89C200123DBE0FB6858
:101B48001B68D3F8B4301B0E03F00103012B0BD133
:101B5800FB681B68D3F8B030DB0F03F00103B3F167
:101B6800004F01D10123FB61FB681B68D3F8B43037
:101B78001B0A03F03F03FA691344FB61FB689A6F81
:101B8800FB68DB6CF96901FB03F39B0013447B6280
:101B980018E0FB681B6DBA689A4209D3FB68D3F852
:101BA8009C3043F02002FB68C3F89C200123A2E08C
:101BB800FB68DA6FFB685B6DB96801FB03F39B0098
:101BC80013447B627B6A1B6803F080427B685A601F
:101BD8007B685B68002B07D17B6A1B689B0CC3F38F
:101BE8000A027B681A6005E07B6A1B6823F0604282
:101BF8007B681A607B6A1B6803F000527B689A60F6
:101C08007B6A1B6803F000427B681A617B6A0433B5
:101C18007B627B6A1B689AB27B68DA617B6A1B68A5
:101C280003F470227B68DA607B6A1B6803F4801215
:101C38007B685A617B6A1B6803F400127B689A61AF
:101C48007B6A1B681B0E03F07F027B681A627B6A43
:101C58001B68DA0F7B685A627B6A04337B627B6A93
:101C68007B6100233B620AE07A693B6A1A4439685F
:101C78003B6A0B4412781A703B6A01333B627B68FB
:101C8800DB681B0C1F4AD35C1A463B6A9342EBD3B2
:101C9800BB68402B05D1FB681B68FA69C3F8A8200C
:101CA8001EE0BB68412B05D1FB681B68FA69C3F8C5
:101CB800B82015E0BB681F2B08D8FB681B680121FA
:101CC800BA6801FA02F2C3F8982009E0BB6803F089
:101CD8001F02FB681B68012101FA02F2C3F89C206D
:101CE800002308E0FB68D3F89C3043F00802FB6847
:101CF800C3F89C20012318462C37BD465DF8047BA9
:101D0800704700BF5C57000880B487B000AFF86028
:101D1800B9607A60FB6893F89830FB75FB7D012BFE
:101D280002D0FB7D022B55D1FB681B689A6DBB68FE
:101D38001340002B08D1FB681B68DA6DFB681B6831
:101D480042F00102DA6514E0FB681B689A6DBB6813
:101D58001340BA689A4208D1FB681B68DA6DFB68C1
:101D68001B6842F00202DA6503E0FB681B68032285
:101D7800DA65BB6803F40073002B09D0FB681B68A5
:101D8800D3F8E010FB681B687A680A43C3F8E020C0
:101D9800BB6803F48063002B09D0FB681B68D3F889
:101DA800E410FB681B687A680A43C3F8E420FB6800
:101DB8001B68596DBA680F4B1340FA6812680B43D9
:101DC80053650D4B5A69BB689B0F0B4913434B6115
:101DD800002308E0FB68D3F89C3043F00202FB685C
:101DE800C3F89C20012318461C37BD465DF8047BC8
:101DF800704700BFFFFFCF3F00A8004080B596B0F6
:101E080000AF78609A4B1B699B077B65984B5B69B1
:101E18009B077A6D13407B657B681B681B6D03F419
:101E280070433B657B681B685B6D3A6D13403B658F
:101E38007B681B681B6D03F00F03FB647B681B68E2
:101E48005B6DFA6C1340FB647B681B681B6D03F0C9
:101E5800F003BB647B681B685B6DBA6C1340BB64A2
:101E68007B681B681B6D03F071537B647B681B6880
:101E78005B6D7A6C13407B647B681B681B6D03F099
:101E880060733B647B681B685B6D3A6C13403B6412
:101E98007B681B685B6DFB637B681B681B6DBB63A2
:101EA800FB6B1B0A03F00103002B10D0BB6B1B0A52
:101EB80003F00103002B0AD07B681B684FF4807283
:101EC8001A656B4B00221A61786800F054FAFB6BB4
:101ED8009B0A03F00103002B1DD0BB6B9B0A03F088
:101EE8000103002B17D07B681B68D3F8DC307B63B9
:101EF8007B681B68D3F8E4307A6B13407B637B689C
:101F08001B684FF480621A65594B00221A61796B7D
:101F1800786800F007FA7B6D002B0DD07B681A6893
:101F2800796D544B0B401365514A7B6D9B0F1361C0
:101F3800796D786800F0C0F93B6D002B0DD07B6897
:101F48001A68396D4B4B0B401365494A3B6D9B0F23
:101F58001361396D786800F0BAF9FB6C002B0DD06D
:101F68007B681A68F96C434B0B401365404AFB6C5D
:101F78009B0F1361F96C7868FEF7BAF9BB6C002BFC
:101F88000DD07B681A68B96C3A4B0B401365384A18
:101F9800BB6C9B0F1361B96C786800F0A3F9FB6BFD
:101FA800DB0A03F00103002B10D0BB6BDB0A03F044
:101FB8000103002B0AD07B681B684FF400621A6586
:101FC8002B4B00221A61786800F097F9FB6B5B0ACB
:101FD80003F00103002B1DD0BB6B5B0A03F0010368
:101FE800002B17D07B681B68D3F8D8303B637B681D
:101FF8001B68D3F8E0303A6B13403B637B681B687F
:102008004FF400721A651A4B00221A61396B78680E
:1020180000F07DF9FB6BDB0C03F00103002B10D003
:10202800BB6BDB0C03F00103002B0AD07B681B6839
:102038004FF400221A650E4B00221A61786800F0EE
:102048007CF9FB6B1B0C03F00103002B16D0BB6B58
:102058001B0C03F00103002B10D07B681B684FF4A6
:1020680080321A65024B00221A61786804E000BFCA
:1020780000A80040FFFFCF3F00F069F9FB6B9B0C05
:1020880003F00103002B10D0BB6B9B0C03F0010382
:10209800002B0AD07B681B684FF480221A65834B9B
:1020A80000221A61786800F05CF9FB6B5B0C03F0A6
:1020B8000103002B15D0BB6B5B0C03F00103002B55
:1020C8000FD07B681B684FF400321A65774B0022EB
:1020D8001A617B68D3F89C3043F080027B68C3F8B0
:1020E8009C203B6C002B0DD07B681A68396C704BB8
:1020F8000B4013656D4A3B6C9B0F1361396C786814
:1021080000F04DF97B6C002B11D07B681A68796C54
:10211800674B0B401365654A7B6C9B0F13617B68AB
:10212800D3F89C207B6C1A437B68C3F89C207B689F
:102138001B68604A934240F0AC807B685B689B6890
:1021480003F00303002B00F0A4807B685B681B6A24
:1021580003F00F03FB627B685B685B6AFA6A1340F3
:10216800FB627B685B681B6A03F03003BB627B68B9
:102178005B685B6ABA6A1340BB627B685B681B6A10
:1021880003F4C0737B627B685B685B6A7A6A13409E
:102198007B627B685B681B6A03F4FC433B627B6879
:1021A8005B685B6A3A6A13403B627B685B681B6AE0
:1021B80003F4F023FB617B685B685B6AFA69134090
:1021C800FB617B685B685B6ABB617B685B681B6AF9
:1021D8007B61FB6A002B07D07B685B68FA6A1A622E
:1021E800F96A786800F0E6F8BB6A002B07D07B68CC
:1021F8005B68BA6A1A62B96A786800F0E6F8BB697F
:102208009B0903F00103002B1AD07B699B0903F09B
:102218000103002B14D07B685B68DB6B1B0C9BB243
:102228003B617B685B68DB6B03F03F03FB607B68AB
:102238005B6840221A62FA683969786800F0D0F859
:102248007B6A002B07D07B685B687A6A1A62796AB6
:10225800786800F0D1F83B6A002B0BD07B685B688C
:102268003A6A1A627B68D3F89C203B6A1A437B68F7
:10227800C3F89C20FB69002B0BD07B685B68FA696C
:102288001A627B68D3F89C20FB691A437B68C3F801
:102298009C207B68D3F89C30002B02D0786800F033
:1022A80074F800BF5837BD4680BD00BF00A8004085
:1022B800FFFFCF3F00A0004080B483B000AF78603C
:1022C800396000BF0C37BD465DF8047B704780B4A9
:1022D80083B000AF7860396000BF0C37BD465DF849
:1022E800047B704780B483B000AF7860396000BF6A
:1022F8000C37BD465DF8047B704780B483B000AFEF
:10230800786000BF0C37BD465DF8047B704780B429
:1023180083B000AF7860396000BF0C37BD465DF808
:10232800047B704780B483B000AF7860396000BF29
:102338000C37BD465DF8047B704780B483B000AFAE
:10234800786000BF0C37BD465DF8047B704780B4E9
:1023580083B000AF786000BF0C37BD465DF8047BE2
:10236800704780B483B000AF786000BF0C37BD46BB
:102378005DF8047B704780B483B000AF786000BF1D
:102388000C37BD465DF8047B704780B483B000AF5E
:10239800786000BF0C37BD465DF8047B704780B499
:1023A80083B000AF7860396000BF0C37BD465DF878
:1023B800047B704780B483B000AF7860396000BF99
:1023C8000C37BD465DF8047B704780B483B000AF1E
:1023D8007860396000BF0C37BD465DF8047B7047F4
:1023E80080B485B000AFF860B9607A6000BF143778
:1023F800BD465DF8047B704780B483B000AF786059
:10240800396000BF0C37BD465DF8047B704700009B
:1024180080B485B000AF78607B685B6BBB607B681D
:102428001B68D3F88420A74B1340BA6891007A68D8
:1024380012680B43C2F884307B681B68D3F8843079
:1024480023F47F017B689B6B1A047B681B680A4333
:10245800C3F884207B689B6BBA681344BB607B68B5
:102468001B68D3F88820974B1340BA6891007A68A4
:1024780012680B43C2F888307B681B68D3F8883031
:1024880023F4FE017B68DB6B1A047B681B680A4334
:10249800C3F888207B68DB6B5B00BA681344BB60B9
:1024A8007B681B68D3F8A020864B1340BA6891005C
:1024B8007A6812680B43C2F8A0307B681B68D3F8AF
:1024C800A03023F4FE017B681B6C1A047B681B6830
:1024D8000A43C3F8A0207B681B6C7A68526C02FB25
:1024E80003F3BA681344BB607B681B68D3F8B02059
:1024F800744B1340BA6891007A6812680B43C2F8AB
:10250800B0307B681B68D3F8B03023F4FE017B68D9
:102518009B6C1A047B681B680A43C3F8B0207B686D
:102528009B6C7A68D26C02FB03F3BA681344BB60F5
:102538007B681B68D3F8AC20624B1340BA689100E3
:102548007A6812680B43C2F8AC307B681B6D7A68F6
:10255800526D02FB03F3BA681344BB607B681B68C7
:10256800D3F8F020574B1340BA6891007A68126884
:102578000B43C2F8F0307B681B68D3F8F03023F4C3
:102588007C117B689B6D1A047B681B680A43C3F83F
:10259800F0207B689B6D5B00BA681344BB607B6866
:1025A8001B68D3F8C020474B1340BA6891007A687B
:1025B80012680B43C2F8C0307B681B68D3F8C03080
:1025C80023F47C117B68DB6D1A047B681B680A4363
:1025D800C3F8C0207B681B68D3F8C03023F07C5157
:1025E8007B681B6E1A067B681B680A43C3F8C02009
:1025F8007B685A6B344B13449A007B68DA667B68B5
:10260800DA6E7B689B6B9B001A447B681A677B6851
:102618001A6F7B68DB6BDB001A447B685A677B6840
:102628005A6F7B681B6C7968496C01FB03F39B004C
:102638001A447B689A677B689A6F7B689B6C796899
:10264800C96C01FB03F39B001A447B68DA677B685B
:10265800DA6F7B681B6D7968496D01FB03F39B009A
:102668001A447B68C3F880207B68D3F880207B6895
:102678009B6DDB001A447B68C3F884207B68D3F821
:1026880084207B68DB6D7968896E01FB03F39B000E
:102698001A447B68C3F888207B68D3F888207B6855
:1026A8001B6E7968896E01FB03F39B001A447B68F3
:1026B800C3F890207B68D3F89030044A934215D928
:1026C80006E000BF0300FFFF002B0010FCD3004012
:1026D8007B68D3F89C3043F020027B68C3F89C20C9
:1026E8007B68032283F89820012310E07B68DB6E67
:1026F800FB6005E0FB6800221A60FB680433FB609E
:102708007B68D3F89030FA689A42F3D300231846CE
:102718001437BD465DF8047B704700BF80B489B0AC
:1027280000AFF860B9607A603B60BB685B68002BFB
:102738000AD1BB681A69BB689B681A43BB681B68E7
:102748009B041343FB610AE0BB681A69BB689B687A
:102758001A43BB681B68134343F08043FB61BB68A3
:102768001B6A1A06BB68DB691A43BB689B691A4374
:10277800BB685B691A43BB68DB6813433B61FB6852
:10278800D3F88420FB689B6E396801FB03F39B0038
:102798001344BB61BB69FA691A60BB690433BB6146
:1027A800BB693A691A60BB690433BB6100237B616A
:1027B80020E07B6903337A6813441B781A067B6927
:1027C800023379680B441B781B041A437B69013375
:1027D80079680B441B781B02134379687A690A44A9
:1027E80012781A43BB691A60BB690433BB617B6901
:1027F80004337B61BB68DB681B0C064AD35C1A4652
:102808007B699342D5D300BF00BF2437BD465DF82E
:10281800047B70475C57000880B58AB000AFF86049
:10282800B9607A60BB683B627B68FB610823FB7513
:10283800404B1B7D012B01D1022376E03D4B012249
:102848001A75BB68B3F1006F06D3BB68B3F1016FAB
:1028580002D20123BB610CE0BB68B3F1016F06D360
:10286800BB68B3F1026F02D20223BB6101E001230E
:102878005BE0304B00229A61B9694CF2503000F0AD
:10288800C1F8034687F8273097F82730002B47D13F
:10289800BB69012B06D1284BDB68274A43F00203AA
:1028A800D36007E0244BD3F80C31234A43F00203EA
:1028B800C2F80C31BFF36F8F00BFBFF34F8F00BF5B
:1028C800FB691A683B6A1A603B6A04333B62FB691E
:1028D8000433FB61FB7D013BFB75FB7D002BEFD1D6
:1028E800BFF36F8F00BFBFF34F8F00BFB9694CF2C2
:1028F800503000F087F8034687F82730BB69012B72
:1029080006D10D4BDB680C4A23F00203D36007E0C5
:10291800094BD3F80C31084A23F00203C2F80C31F2
:10292800044B00221A7597F8273018462837BD46F9
:1029380080BD00BF640300240020005280B400AFB3
:10294800184BDB6803F00103002B0DD0154B164A1A
:102958005A60144B154A5A60124BDB6803F00103A6
:10296800002B01D0012318E00E4BD3F80C3103F0F3
:102978000103002B10D00B4B0B4AC3F80421094B61
:102988000A4AC3F80421074BD3F80C3103F00103BA
:10299800002B01D0012300E000231846BD465DF856
:1029A800047B70470020005223016745AB89EFCDB7
:1029B80080B400AF124BDB68114A43F00103D360C7
:1029C8000F4BDB6803F00103002B01D1012311E059
:1029D8000B4BD3F80C310A4A43F00103C2F80C310F
:1029E800074BD3F80C3103F00103002B01D101236D
:1029F80000E000231846BD465DF8047B704700BF21
:102A08000020005280B586B000AF7860396004239A
:102A18007B6100233B61FEF727FCF8603B68022BD3
:102A280013D1414B7B6110E07B68B3F1FF3F0CD0C1
:102A3800FEF71AFC0246FB68D31A7A689A4202D358
:102A48007B68002B01D103236AE07A69374B134076
:102A58007A699A420AD1364B1A697B6913407A69B6
:102A68009A420CBF01230023DBB20CE0304BD3F8B1
:102A78001031DA437B69134023F00043002B0CBF6D
:102A880001230023DBB2002BCED13B68012B05D1FB
:102A9800274B1A69274B13403B6107E0244BD3F8B7
:102AA8001021244B134043F000433B613B6923F062
:102AB8000043002B17D0204B9A693B6913431E4AE9
:102AC80093613A69194B13403A699A4203D1184AFB
:102AD8003B69536105E0164A3B6923F00043C2F89D
:102AE800143101231CE03B68012B0BD1104B1B69EF
:102AF80003F48033B3F5803F11D10D4B4FF480328E
:102B08005A610CE00A4BD3F8103103F48033B3F563
:102B1800803F04D1064B4FF48032C3F814210023C0
:102B280018461837BD4680BD040000800F00EF1F0F
:102B3800002000520000EE176403002480B584B022
:102B480000AF786039600023FB735E4B1B7D012B5F
:102B580001D10223B2E05B4B01221A75594B0022C6
:102B68009A617B685B6803F00103002B09D001219F
:102B78004CF25030FFF746FF0346002B01D00123EB
:102B8800FB737B685B6803F00203002B09D002210A
:102B98004CF25030FFF736FF0346002B01D00123DB
:102BA800FB73FB7B002B40F085807B681B68012B47
:102BB80036D17B681A697B685B681946104600F055
:102BC80087F87B685B6803F00103002B0FD00121B5
:102BD8004CF25030FFF716FF0346002B01D00123BB
:102BE800FB73394BDB68384A23F00803D3607B68F2
:102BF8005B6803F00203002B5CD002214CF25030DA
:102C0800FFF700FF0346002B01D00123FB732E4B77
:102C1800D3F80C312C4A23F00803C2F80C3149E0F0
:102C28003B684FF0FF321A607B689B68BB6039E0F5
:102C38007B6859687B681B691A46B86800F0B2F867
:102C48007B685B6803F00103002B0CD001214CF278
:102C58005030FFF7D7FE0346FB731B4BDA681A495F
:102C68001A4B1340CB607B685B6803F00203002BB0
:102C78000ED002214CF25030FFF7C4FE0346FB731E
:102C8800114BD3F80C211049104B1340C1F80C31EB
:102C9800FB7B002B03D03B68BA681A600AE0BB686C
:102CA8000133BB607B68DA687B689B681344BA6849
:102CB8009A42BDD3034B00221A75FB7B1846103786
:102CC800BD4680BD6403002400200052FBF8FFFFCE
:102CD80080B483B000AF786039603B6803F00303C9
:102CE800032B22D12E4BDB682D4A23F03003D3600F
:102CF8002B4BD3F80C312A4A23F03003C2F80C319D
:102D0800274BDA6826497B681343CB60244BD3F8FA
:102D18000C2123497B681343C1F80C31204B9B6974
:102D28001F4A43F01003936133E03B6803F001034B
:102D3800002B11D01A4BDB68194A23F03003D360FB
:102D4800174BDA6816497B681343CB60144BDB6872
:102D5800134A43F08803D3603B6803F00203002B57
:102D680017D00F4BD3F80C310D4A23F03003C2F8BB
:102D78000C310B4BD3F80C2109497B681343C1F87C
:102D88000C31074BD3F80C31054A43F08803C2F8DD
:102D98000C3100BF0C37BD465DF8047B704700BF9F
:102DA8000020005280B485B000AFF860B9607A6046
:102DB800BB6803F00103002B10D0184BDB68174ADF
:102DC80023F4E663D360154BDA68FB6819027B6865
:102DD8000B431343114A43F08403D360BB6803F0E9
:102DE8000203002B14D00D4BD3F80C310B4A23F4FB
:102DF800E663C2F80C31094BD3F80C21FB681902C1
:102E08007B680B431343054A43F08403C2F80C3133
:102E180000BF1437BD465DF8047B704700200052A0
:102E280080B489B000AF786039600023FB61894BBA
:102E38007B6194E13B681A680121FB6901FA03F39D
:102E480013403B613B69002B00F086813B685B685F
:102E580003F00303012B05D03B685B6803F0030311
:102E6800022B30D17B689B68BB61FB695B00032246
:102E780002FA03F3DB43BA691340BB613B68DA68C3
:102E8800FB695B0002FA03F3BA691343BB617B6811
:102E9800BA699A607B685B68BB610122FB6902FAC8
:102EA80003F3DB43BA691340BB613B685B681B09EA
:102EB80003F00102FB6902FA03F3BA691343BB6129
:102EC8007B68BA695A603B685B6803F00303032BAD
:102ED80017D07B68DB68BB61FB695B00032202FAE1
:102EE80003F3DB43BA691340BB613B689A68FB692B
:102EF8005B0002FA03F3BA691343BB617B68BA69E2
:102F0800DA603B685B6803F00303022B23D1FB699B
:102F1800DA087B68083253F82230BB61FB6903F09A
:102F280007039B000F2202FA03F3DB43BA6913403D
:102F3800BB613B681A69FB6903F007039B0002FA4F
:102F480003F3BA691343BB61FB69DA087B6808328B
:102F5800B96943F822107B681B68BB61FB695B0099
:102F6800032202FA03F3DB43BA691340BB613B68EF
:102F78005B6803F00302FB695B0002FA03F3BA69BA
:102F88001343BB617B68BA691A603B685B6803F4EA
:102F98004033002B00F0E0802F4BD3F8F4302E4A5A
:102FA80043F00203C2F8F4302B4BD3F8F43003F0AB
:102FB8000203FB60FB68294AFB699B08023352F84D
:102FC8002330BB61FB6903F003039B000F2202FA65
:102FD80003F3DB43BA691340BB617B68204A934221
:102FE80052D07B681F4A934231D07B681E4A934275
:102FF8002BD07B681D4A934225D07B681C4A93429C
:103008001FD07B681B4A934219D07B681A4A9342A7
:1030180013D07B68194A93420DD07B68184A9342B3
:1030280007D07B68174A934201D109232DE00A2370
:103038002BE0082329E0072327E0062325E00523C2
:1030480023E0042321E003231FE002231DE00123E2
:103058001BE000BF800000580044025800040058DC
:10306800000002580004025800080258000C0258D8
:10307800001002580014025800180258001C025888
:1030880000200258002402580023FA6902F00302C3
:1030980092009340BA691343BB613849FB699B08A6
:1030A8000233BA6941F823204FF0B0431B68BB6173
:1030B8003B69DB43BA691340BB613B685B6803F457
:1030C8008013002B03D0BA693B691343BB614FF0EF
:1030D800B042BB6913604FF0B0435B68BB613B69AA
:1030E800DB43BA691340BB613B685B6803F40013B8
:1030F800002B03D0BA693B691343BB614FF0B04260
:10310800BB6953607B695B68BB613B69DB43BA6938
:103118001340BB613B685B6803F40033002B03D0AA
:10312800BA693B691343BB617B69BA695A607B69B9
:103138001B68BB613B69DB43BA691340BB613B68F1
:103148005B6803F48033002B03D0BA693B691343EF
:10315800BB617B69BA691A60FB690133FB613B6833
:103168001A68FB6922FA03F3002B7FF463AE00BFF1
:1031780000BF2437BD465DF8047B70470004005843
:1031880080B487B000AF7860396000237B61754BED
:103198003B61D9E001227B6902FA03F33A681340E4
:1031A800FB60FB68002B00F0CC806F4A7B699B08B2
:1031B800023352F82330BB607B6903F003039B00A2
:1031C8000F2202FA03F3BA681340BB607B68674AB0
:1031D800934237D07B68664A934231D07B68654A10
:1031E80093422BD07B68644A934225D07B68634A1C
:1031F80093421FD07B68624A934219D07B68614A28
:10320800934213D07B68604A93420DD07B685F4A33
:10321800934207D07B685E4A934201D1092312E0AA
:103228000A2310E008230EE007230CE006230AE037
:10323800052308E0042306E0032304E0022302E058
:10324800012300E000237A6902F003029200934010
:10325800BA689A4236D13B691A68FB68DB431A4060
:103268003B691A603B695A68FB68DB431A403B6953
:103278005A604FF0B0435A68FB68DB434FF0B041E7
:1032880013404B604FF0B0431A68FB68DB434FF0C4
:10329800B04113400B607B6903F003039B000F22CE
:1032A80002FA03F3BB60304A7B699B08023352F889
:1032B8002310BB68DA432C487B699B080A40023319
:1032C80040F823207B681A687B695B00032101FAB8
:1032D80003F31A437B681A607B69DA087B68083253
:1032E80053F822107B6903F007039B000F2202FAB0
:1032F80003F3DB437A69D20819407B68083243F844
:1033080022107B68DA687B695B00032101FA03F30A
:10331800DB431A407B68DA607B685A6801217B6965
:1033280001FA03F3DB431A407B685A607B689A68AA
:103338007B695B00032101FA03F3DB431A407B68D6
:103348009A607B6901337B613A687B6922FA03F3EF
:10335800002B7FF41FAF00BF00BF1C37BD465DF8D0
:10336800047B704780000058000400580000025891
:103378000004025800080258000C025800100258B5
:103388000014025800180258001C02580020025865
:103398000024025880B584B000AF7860194BDB6810
:1033A80003F00403042B0AD0164BDB6803F0070371
:1033B8007A689A4201D001231FE000231DE0114BD7
:1033C800DB6823F007020F497B681343CB60FDF7E6
:1033D8004BFFF86009E0FDF747FF0246FB68D31A88
:1033E800B3F57A7F01D9012307E0064B5B6803F444
:1033F8000053B3F5005FEED1002318461037BD46E1
:1034080080BD00BF0048025880B582B000AF894B2C
:103418001B6803F00F03062B0FD8864B1B6823F09D
:103428000F03844A43F007031360824B1B6803F0C1
:103438000F03072B01D00123F7E0FDF715FF786094
:103448007D4B1B687C4A43F00103136008E0FDF7DD
:103458000BFF02467B68D31A022B01D90323E4E051
:10346800754B1B6803F00403002BF0D0724B5B68AC
:10347800714A43F0804353606F4B00221A616F4BCF
:103488006F4A1A606F4B6E4A1A606F4B1B6818467A
:10349800FDF7A0FE0346002B01D00123C5E0FDF790
:1034A800E3FE78600AE0FDF7DFFE02467B68D31A88
:1034B80041F28832934201D90323B6E05E4B1B697F
:1034C80003F03803002BEED1FDF7CEFE78605A4B9F
:1034D8001A6859495D4B13400B6008E0FDF7C4FEBC
:1034E80002467B68D31A642B01D903239DE0524B13
:1034F8001B6803F40033002BF0D1FDF7B5FE7860AC
:103508004D4B1B684C4A23F08073136008E0FDF7AD
:10351800ABFE02467B68D31A022B01D9032384E051
:10352800454B1B6803F00073002BF0D1FDF79CFEA0
:103538007860414B1B68404A23F08063136008E0C1
:10354800FDF792FE02467B68D31A022B01D90323AA
:103558006BE0394B1B6803F00063002BF0D1FDF7DB
:1035680083FE7860344B1B68334A23F08053136022
:1035780008E0FDF779FE02467B68D31A022B01D9D1
:10358800032352E02C4B1B6803F00053002BF0D1AF
:10359800294B00229A61284B0022DA61264B00222F
:1035A8001A62254B2A4A9A62234B2A4ADA62224B2C
:1035B800294A1A63204B00225A631F4B264A9A63F2
:1035C8001D4B0022DA631C4B234A1A641A4B002253
:1035D8005A64194B1B68184A23F480231360164B4E
:1035E80000221A66144B4FF0FF329A66124BD3F83A
:1035F800D030114A43F48033C2F8D0300D4B1B68E9
:1036080003F00803002B0FD00A4B1B6823F00F03AD
:10361800084A43F007031360064B1B6803F00F03C7
:10362800072B01D0012300E0002318460837BD46C8
:1036380080BD00BF00200052004402580000002452
:103648000090D003040000240800002445EDF6FF94
:10365800000202020000FF018002010180B58CB067
:1036680000AF78607B68002B02D1012300F01DBCFD
:103678007B681B6803F00103002B00F08780994BDF
:103688001B6903F03803FB62964B9B6ABB62FB6ABB
:10369800102B07D0FB6A182B10D1BB6A03F0030369
:1036A800022B0BD18F4B1B6803F40033002B6CD01B
:1036B8007B685B68002B68D10123F6E37B685B6855
:1036C800B3F5803F06D1874B1B68864A43F48033A5
:1036D80013602EE07B685B68002B0CD1814B1B6864
:1036E800804A23F4803313607E4B1B687D4A23F4A1
:1036F800802313601DE07B685B68B3F5A02F0CD1B5
:10370800784B1B68774A43F480231360754B1B681A
:10371800744A43F4803313600BE0724B1B68714AA0
:1037280023F4803313606F4B1B686E4A23F48023A5
:1037380013607B685B68002B13D0FDF795FD7862FA
:1037480008E0FDF791FD02467B6AD31A642B01D984
:103758000323AAE3634B1B6803F40033002BF0D068
:1037680014E0FDF781FD786208E0FDF77DFD024673
:103778007B6AD31A642B01D9032396E3594B1B6840
:1037880003F40033002BF0D100E000BF7B681B6816
:1037980003F00203002B00F0CB80524B1B6903F0AF
:1037A80038033B624F4B9B6AFB613B6A002B07D097
:1037B8003B6A182B56D1FB6903F00303002B51D148
:1037C800484B1B6803F00403002B05D07B68DB68BB
:1037D800002B01D1012368E3424B1B6823F0190237
:1037E8007B68DB683F4913430B60FDF73DFD78625A
:1037F80008E0FDF739FD02467B6AD31A022B01D98E
:10380800032352E3374B1B6803F00403002BF0D06B
:10381800FDF75AFD034641F20302934217D87B682D
:103828001B69402B08D12F4B5B6823F47C332D4A4E
:1038380043F4003353607BE02A4B5B6823F47C320B
:103848007B681B691B03274913434B6070E0254BBA
:103858005B6823F0FE427B681B691B062149134302
:103868004B6065E07B68DB68002B48D01D4B1B680C
:1038780023F019027B68DB681A4913430B60FDF7D4
:10388800F3FC786208E0FDF7EFFC02467B6AD31A86
:10389800022B01D9032308E3124B1B6803F004032E
:1038A800002BF0D0FDF710FD034641F203029342CE
:1038B8001AD87B681B69402B08D10A4B5B6823F434
:1038C8007C33084A43F40033536031E0054B5B68AE
:1038D80023F47C327B681B691B03024913434B604A
:1038E80026E000BF004402589A4B5B6823F0FE4272
:1038F8007B681B691B06974913434B6018E0954B7F
:103908001B68944A23F001031360FDF7ADFC78624D
:1039180008E0FDF7A9FC02467B6AD31A022B01D9FD
:103928000323C2E28B4B1B6803F00403002BF0D186
:103938007B681B6803F01003002B00F0A980854BFF
:103948001B6903F03803BB61824B9B6A7B61BB69CF
:10395800082B07D0BB69182B3AD17B6903F0030306
:10396800012B35D17B4B1B6803F48073002B05D0EA
:103978007B68DB69802B01D0012396E2FDF7A4FC6C
:10398800034641F20302934217D87B681B6A202B37
:1039980008D1704B5B6823F0F8436E4A43F08043CC
:1039A800536075E06B4B5B6823F0F8427B681B6AD9
:1039B8009B06684913434B606AE0664BDB6823F05B
:1039C8007C527B681B6A1B0662491343CB605FE02D
:1039D8007B68DB69002B42D05E4B1B685D4A43F075
:1039E80080031360FDF740FC786208E0FDF73CFCBB
:1039F80002467B6AD31A022B01D9032355E2554BA1
:103A08001B6803F48073002BF0D0FDF75DFC0346C0
:103A180041F20302934217D87B681B6A202B08D116
:103A28004C4B5B6823F0F8434A4A43F080435360A9
:103A38002EE0484B5B6823F0F8427B681B6A9B06C4
:103A4800444913434B6023E0424BDB6823F07C522C
:103A58007B681B6A1B063F491343CB6018E03D4B4C
:103A68001B683C4A23F080031360FDF7FDFB786276
:103A780008E0FDF7F9FB02467B6AD31A022B01D94D
:103A8800032312E2334B1B6803F48073002BF0D13D
:103A98007B681B6803F00803002B36D07B685B69E2
:103AA800002B19D02B4B5B6F2A4A43F00103536755
:103AB800FDF7DAFB786208E0FDF7D6FB02467B6A81
:103AC800D31A022B01D90323EFE1224B5B6F03F0DA
:103AD8000203002BF0D018E01E4B5B6F1D4A23F049
:103AE80001035367FDF7C0FB786208E0FDF7BCFBF4
:103AF80002467B6AD31A022B01D90323D5E1154B61
:103B08005B6F03F00203002BF0D17B681B6803F0A6
:103B18002003002B39D07B689B69002B1CD00D4BF0
:103B28001B680C4A43F480531360FDF79DFB7862D1
:103B380008E0FDF799FB02467B6AD31A022B01D9EC
:103B48000323B2E1034B1B6803F40053002BF0D0AE
:103B58001BE000BF004402589B4B1B689A4A23F4A1
:103B680080531360FDF780FB786208E0FDF77CFB6B
:103B780002467B6AD31A022B01D9032395E1924BA3
:103B88001B6803F40053002BF0D17B681B6803F01B
:103B98000403002B00F081808C4B1B688B4A43F494
:103BA80080731360FDF760FB786208E0FDF75CFB4B
:103BB80002467B6AD31A642B01D9032375E1834B30
:103BC8001B6803F48073002BF0D07B689B68012B83
:103BD80006D17D4B1B6F7C4A43F0010313672DE030
:103BE8007B689B68002B0CD1774B1B6F764A23F0C0
:103BF80001031367744B1B6F734A23F004031367A5
:103C08001CE07B689B68052B0CD16F4B1B6F6E4AC1
:103C180043F0040313676C4B1B6F6B4A43F00103BB
:103C280013670BE0684B1B6F674A23F001031367A8
:103C3800654B1B6F644A23F0040313677B689B681A
:103C4800002B15D0FDF710FB78620AE0FDF70CFB9E
:103C580002467B6AD31A41F28832934201D9032380
:103C680023E1594B1B6F03F00203002BEED014E045
:103C7800FDF7FAFA78620AE0FDF7F6FA02467B6A7F
:103C8800D31A41F28832934201D903230DE14E4BF6
:103C98001B6F03F00203002BEED17B685B6A002BDD
:103CA80000F00281484B1B6903F03803182B00F021
:103CB800BD807B685B6A022B40F09E80424B1B688C
:103CC800414A23F080731360FDF7CEFA786208E06A
:103CD800FDF7CAFA02467B6AD31A022B01D90323DD
:103CE800E3E0394B1B6803F00073002BF0D1364B2F
:103CF8009A6A374B13407A68916A7A68D26A1201D5
:103D08000A43314913438B627B681B6B013BC3F346
:103D180008027B685B6B013B5B029BB21A437B68C2
:103D28009B6B013B1B0403F4FE031A437B68DB6BAC
:103D3800013B1B0603F0FE43234913430B63224B4D
:103D4800DB6A214A23F00103D3621F4B5A6B214BD4
:103D580013407A68926CD2001B4913434B631A4B89
:103D6800DB6A23F00C027B681B6C17491343CB6298
:103D7800154BDB6A23F002027B685B6C1249134324
:103D8800CB62114BDB6A104A43F48033D3620E4B8B
:103D9800DB6A0D4A43F40033D3620B4BDB6A0A4AF1
:103DA80043F48023D362084BDB6A074A43F00103DC
:103DB800D362054B1B68044A43F080731360FDF718
:103DC80053FA786211E000BF0044025800480258D4
:103DD8000CFCFFFF0700FFFFFDF746FA02467B6A6F
:103DE800D31A022B01D903235FE0324B1B6803F07F
:103DF8000073002BF0D057E02E4B1B682D4A23F0A0
:103E080080731360FDF730FA786208E0FDF72CFA4A
:103E180002467B6AD31A022B01D9032345E0254BBE
:103E28001B6803F00073002BF0D13DE0214B9B6A27
:103E38003B61204B1B6BFB607B685B6A012B31D0BD
:103E48003B6903F003027B689B6A9A422AD13B696B
:103E58001B0903F03F027B68DB6A9A4222D1FB68A8
:103E6800C3F308027B681B6B013B9A421AD1FB68BB
:103E78005B0A03F07F027B685B6B013B9A4211D1BE
:103E8800FB681B0C03F07F027B689B6B013B9A422B
:103E980008D1FB681B0E03F07F027B68DB6B013BDC
:103EA8009A4201D0012300E0002318463037BD466E
:103EB80080BD00BF0044025880B586B000AF78606E
:103EC80039607B68002B01D101239CE18A4B1B6878
:103ED80003F00F033A689A4210D9874B1B6823F006
:103EE8000F0285493B6813430B60834B1B6803F043
:103EF8000F033A689A4201D0012384E17B681B686A
:103F080003F00403002B10D07B681A697B4B9B6974
:103F180003F070039A4208D9784B9B6923F070022A
:103F28007B681B69754913438B617B681B6803F0C9
:103F38000803002B10D07B685A69704BDB6903F0CB
:103F480070039A4208D96D4BDB6923F070027B68D5
:103F58005B696A491343CB617B681B6803F01003F4
:103F6800002B10D07B689A69644BDB6903F4E0632B
:103F78009A4208D9614BDB6923F4E0627B689B694C
:103F88005E491343CB617B681B6803F02003002B59
:103F980010D07B68DA69594B1B6A03F070039A42A8
:103FA80008D9564B1B6A23F070027B68DB695349BA
:103FB80013430B627B681B6803F00203002B10D0CD
:103FC8007B68DA684D4B9B6903F00F039A4208D966
:103FD8004A4B9B6923F00F027B68DB684749134310
:103FE8008B617B681B6803F00103002B55D0434BA2
:103FF8009B6923F470627B689B68404913438B611B
:104008007B685B68022B07D13C4B1B6803F40033C9
:10401800002B21D10123F6E07B685B68032B07D1D5
:10402800364B1B6803F00073002B15D10123EAE01F
:104038007B685B68012B07D1304B1B6803F48073E6
:10404800002B09D10123DEE02C4B1B6803F004038D
:10405800002B01D10123D6E0284B1B6923F007026E
:104068007B685B68254913430B61FDF7FDF87861B0
:104078000AE0FDF7F9F802467B69D31A41F2883263
:10408800934201D90323BEE01C4B1B6903F038029D
:104098007B685B68DB009A42EBD17B681B6803F0A6
:1040A8000203002B10D07B68DA68144B9B6903F07D
:1040B8000F039A4208D2114B9B6923F00F027B68C9
:1040C800DB680E4913438B610B4B1B6803F00F032E
:1040D8003A689A4214D2084B1B6823F00F0206492B
:1040E8003B6813430B60044B1B6803F00F033A68EB
:1040F8009A4205D0012386E000200052004402586D
:104108007B681B6803F00403002B10D07B681A69D6
:104118003F4B9B6903F070039A4208D23C4B9B6962
:1041280023F070027B681B69394913438B617B68F4
:104138001B6803F00803002B10D07B685A69344BC6
:10414800DB6903F070039A4208D2314BDB6923F034
:1041580070027B685B692E491343CB617B681B68DF
:1041680003F01003002B10D07B689A69284BDB6999
:1041780003F4E0639A4208D2254BDB6923F4E0623A
:104188007B689B6922491343CB617B681B6803F0FA
:104198002003002B10D07B68DA691D4B1B6A03F0E3
:1041A80070039A4208D21A4B1B6A23F070027B688C
:1041B800DB69174913430B6200F034F80246144BCD
:1041C8009B691B0A03F00F031249CB5C03F01F0322
:1041D80022FA03F33B610E4B9B6903F00F030D4A70
:1041E800D35C03F01F033A6922FA03F30A4A136007
:1041F8000A4A3B6913600A4B1B681846FCF7EAFF3A
:104208000346FB73FB7B18461837BD4680BD00BFCD
:10421800004402584C570008040000240000002401
:104228000800002480B489B000AFB34B1B6903F0C9
:104238003803182B00F2558101A252F823F000BF71
:10424800AD420008EB440008EB440008EB440008CA
:10425800EB440008EB440008EB440008EB4400087A
:10426800D3420008EB440008EB440008EB44000884
:10427800EB440008EB440008EB440008EB4400085A
:10428800D9420008EB440008EB440008EB4400085E
:10429800EB440008EB440008EB440008EB4400083A
:1042A800DF420008944B1B6803F02003002B09D061
:1042B800914B1B68DB0803F00303904A22FA03F3CF
:1042C800BB6111E18D4BBB610EE18D4BBB610BE115
:1042D8008C4BBB6108E1884B9B6A03F003037B614D
:1042E800854B9B6A1B0903F03F033B61824BDB6AEA
:1042F80003F00103FB60804B5B6BDB08C3F30C032B
:10430800FA6802FB03F307EE903AF8EE677AC7ED16
:10431800027A3B69002B00F0E1807B69022B00F0F8
:1043280083807B69022B00F2A1807B69002B03D07C
:104338007B69012B56D099E06F4B1B6803F0200373
:10434800002B2DD06C4B1B68DB0803F003036B4A72
:1043580022FA03F37B607B6807EE903AF8EE676A0F
:104368003B6907EE903AF8EE677A86EEA77A624BD9
:104378001B6BC3F3080307EE903AF8EE676A97EDF4
:10438800026ADFED615AC6EE257A76EEA77AF7EE75
:10439800006A77EEA67A67EE277AC7ED077A87E094
:1043A8003B6907EE903AF8EE677ADFED586A86EED9
:1043B800A77A514B1B6BC3F3080307EE903AF8EE4C
:1043C800676A97ED026ADFED505AC6EE257A76EEF7
:1043D800A77AF7EE006A77EEA67A67EE277AC7ED36
:1043E800077A65E03B6907EE903AF8EE677ADFED09
:1043F800486A86EEA77A404B1B6BC3F3080307EEA7
:10440800903AF8EE676A97ED026ADFED3F5AC6EE1A
:10441800257A76EEA77AF7EE006A77EEA67A67EE47
:10442800277AC7ED077A43E03B6907EE903AF8EE42
:10443800677ADFED386A86EEA77A2F4B1B6BC3F3DA
:10444800080307EE903AF8EE676A97ED026ADFED27
:104458002E5AC6EE257A76EEA77AF7EE006A77EE40
:10446800A67A67EE277AC7ED077A21E03B6907EE5F
:10447800903AF8EE677ADFED266A86EEA77A1E4B49
:104488001B6BC3F3080307EE903AF8EE676A97EDE3
:10449800026ADFED1D5AC6EE257A76EEA77AF7EEA8
:1044A800006A77EEA67A67EE277AC7ED077A00BF2B
:1044B800114B1B6B5B0A03F07F0301333B603B68C6
:1044C80007EE903AB8EE677AD7ED076AC6EE877AB4
:1044D800FCEEE77A17EE903ABB6105E00023BB617A
:1044E80002E0074BBB6100BFBB6918462437BD46D5
:1044F8005DF8047B704700BF004402580090D00369
:1045080000093D0040787D01000000460024744CFD
:104518000024744A20BCBE4B80B586B000AF7860DA
:104528000023FB750023BB757B681B6803F00063E1
:10453800002B3FD07B685B6EB3F5401F2AD0B3F5E4
:10454800401F24D8B3F5001F18D0B3F5001F1ED89C
:10455800002B03D0B3F5801F07D018E0A34BDB6A0C
:10456800A24A43F40033D36215E07B680433022186
:10457800184600F017FF0346FB750CE07B682433F0
:104588000221184600F0C0FF0346FB7503E0012333
:10459800FB7500E000BFFB7D002B09D1934B1B6D21
:1045A80023F440127B685B6E904913430B6501E06E
:1045B800FB7DBB757B681B6803F48073002B3DD0C3
:1045C8007B685B6D042B26D801A252F823F000BF4C
:1045D800ED450008FB4500080D4600082546000883
:1045E80025460008814BDB6A804A43F40033D362D6
:1045F80015E07B6804330021184600F0D3FE03461B
:10460800FB750CE07B6824330021184600F07CFF22
:104618000346FB7503E00123FB7500E000BFFB7D4B
:10462800002B09D1714B1B6D23F007027B685B6D72
:104638006E4913430B6501E0FB7DBB757B681B6806
:1046480003F40073002B42D07B689B6DB3F5807F29
:104658002BD0B3F5807F25D8C02B28D0C02B21D8EC
:10466800802B16D0802B1DD8002B02D0402B07D0D2
:1046780018E05E4BDB6A5D4A43F40033D36217E00F
:104688007B6804330021184600F08CFE0346FB7556
:104698000EE07B6824330021184600F035FF0346FE
:1046A800FB7505E00123FB7502E000BF00E000BFD9
:1046B800FB7D002B09D14D4B1B6D23F4E0727B6809
:1046C8009B6D4A4913430B6501E0FB7DBB757B6815
:1046D8001B6803F48063002B49D07B68D3F8A430AF
:1046E800B3F5000F30D0B3F5000F2AD8B3F5C00FDB
:1046F8002CD0B3F5C00F24D8B3F5800F18D0B3F57C
:10470800800F1ED8002B03D0B3F5001F07D018E088
:10471800364BDB6A354A43F40033D36217E07B68D3
:1047280004330021184600F03DFE0346FB750EE0F9
:104738007B6824330021184600F0E6FE0346FB752B
:1047480005E00123FB7502E000BF00E000BFFB7D30
:10475800002B0AD1254B9B6D23F460027B68D3F8AC
:10476800A430224913438B6501E0FB7DBB757B6850
:104778001B6803F40063002B4BD07B68D3F8A83088
:10478800B3F1806F30D0B3F1806F2AD8B3F1407F96
:104798002ED0B3F1407F24D8B3F1007F18D0B3F105
:1047A800007F1ED8002B03D0B3F1807F07D018E01C
:1047B8000E4BDB6A0D4A43F40033D36219E07B6881
:1047C80004330021184600F0EDFD0346FB7510E0A8
:1047D8007B6824330021184600F096FE0346FB75DB
:1047E80007E00123FB7504E000BF02E00044025823
:1047F80000BFFB7D002B0AD1994B9B6D23F0E06233
:104808007B68D3F8A830964913438B6501E0FB7D9C
:10481800BB757B681B6803F00073002B32D07B6884
:104828009B6C302B1CD0302B17D8202B0CD0202B76
:1048380013D8002B16D0102B0FD1894BDB6A884A6E
:1048480043F40033D3620EE07B6804330221184638
:1048580000F0A8FD0346FB7505E00123FB7502E0A7
:1048680000BF00E000BFFB7D002B09D17C4BDB6C57
:1048780023F030027B689B6C79491343CB6401E0D9
:10488800FB7DBB757B681B6803F48053002B47D006
:104898007B68DB6DB3F5804F30D0B3F5804F2AD8F5
:1048A800B3F5405F2CD0B3F5405F24D8B3F5005F73
:1048B80018D0B3F5005F1ED8002B03D0B3F5805F86
:1048C80007D018E0664BDB6A654A43F40033D362CD
:1048D80017E07B6804330021184600F063FD0346A7
:1048E800FB750EE07B6824330021184600F00CFEAF
:1048F8000346FB7505E00123FB7502E000BF00E0FD
:1049080000BFFB7D002B09D1554B1B6D23F4E04202
:104918007B68DB6D524913430B6501E0FB7DBB757A
:104928007B681B6803F40053002B49D07B681B6E1F
:10493800B3F5A02F2ED0B3F5A02F28D8B3F5802F2C
:104948002AD0B3F5802F22D8B3F5403F26D0B3F54F
:10495800403F1CD8B3F5003F10D0B3F5003F16D840
:10496800002B1DD0B3F5803F11D17B6804330121A2
:10497800184600F017FD0346FB7512E07B682433E8
:104988000121184600F0C0FD0346FB7509E001232C
:10499800FB7506E000BF04E000BF02E000BF00E0D6
:1049A80000BFFB7D002B09D12D4B1B6D23F4E022AA
:1049B8007B681B6E2A4913430B6501E0FB7DBB75C1
:1049C8007B681B6803F48043002B4DD07B68D3F8C9
:1049D800AC30B3F1A04F2ED0B3F1A04F28D8B3F12B
:1049E800804F2AD0B3F1804F22D8B3F1405F26D050
:1049F800B3F1405F1CD8B3F1005F10D0B3F1005F92
:104A080016D8002B1DD0B3F1805F11D17B68043319
:104A18000121184600F0C6FC0346FB7512E07B68CE
:104A280024330121184600F06FFD0346FB7509E0A9
:104A38000123FB7506E000BF04E000BF02E000BFF1
:104A480000E000BFFB7D002B0CD1054B9B6D23F0D4
:104A5800E0427B68D3F8AC30014913438B6503E02F
:104A680000440258FB7DBB757B681B6803F4004358
:104A7800002B2FD07B68DB6EB3F1005F0ED0B3F153
:104A8800005F14D8002B15D0B3F1805F0FD1AF4B66
:104A9800DB6AAE4A43F40033D3620CE07B6804332C
:104AA8000121184600F07EFC0346FB7503E0012354
:104AB800FB7500E000BFFB7D002B09D1A34B1B6DEC
:104AC80023F040527B68DB6EA04913430B6501E07D
:104AD800FB7DBB757B681B6803F08073002B32D0AD
:104AE8007B685B6C032B1BD801A252F823F000BF34
:104AF8002F4B0008094B0008174B00082F4B0008E4
:104B0800924BDB6A914A43F40033D3620CE07B6832
:104B180004330221184600F045FC0346FB7503E008
:104B28000123FB7500E000BFFB7D002B09D1874BFB
:104B3800DB6C23F003027B685B6C84491343CB6412
:104B480001E0FB7DBB757B681B6803F48003002BC9
:104B580000F086807E4B1B687D4A43F480731360A7
:104B6800FCF782FB386109E0FCF77EFB02463B69F3
:104B7800D31A642B02D90323FB7505E0744B1B6819
:104B880003F48073002BEFD0FB7D002B66D16F4BB5
:104B98001A6F7B68D3F8B030534003F44073002B8E
:104BA80013D06A4B1B6F23F44073FB60674B1B6F7A
:104BB800664A43F480331367644B1B6F634A23F4DC
:104BC80080331367614AFB6813677B68D3F8B0309A
:104BD800B3F5807F15D1FCF747FB38610BE0FCF794
:104BE80043FB02463B69D31A41F28832934202D909
:104BF8000323FB7505E0554B1B6F03F00203002BE5
:104C0800EDD0FB7D002B26D17B68D3F8B03003F4C0
:104C18004073B3F5407F0DD14C4B1B6923F47C5294
:104C28007B68D3F8B03019094A4B0B404749134306
:104C38000B6105E0454B1B69444A23F47C5313611F
:104C4800424B1A6F7B68D3F8B030C3F30B033F496C
:104C580013430B6704E0FB7DBB7501E0FB7DBB756F
:104C68007B681B6803F00103002B00F085807B68DC
:104C78009B6F282B66D801A252F823F0614D0008DB
:104C88004D4D00084D4D00084D4D00084D4D000894
:104C98004D4D00084D4D00084D4D0008294D0008A8
:104CA8004D4D00084D4D00084D4D00084D4D000874
:104CB8004D4D00084D4D00084D4D00083B4D000876
:104CC8004D4D00084D4D00084D4D00084D4D000854
:104CD8004D4D00084D4D00084D4D0008614D000830
:104CE8004D4D00084D4D00084D4D00084D4D000834
:104CF8004D4D00084D4D00084D4D0008614D000810
:104D08004D4D00084D4D00084D4D00084D4D000813
:104D18004D4D00084D4D00084D4D0008614D0008EF
:104D28007B6804330121184600F03CFB0346FB7501
:104D380013E07B6824330121184600F0E5FB0346A5
:104D4800FB750AE00123FB7507E000BF0044025829
:104D580000480258CFFFFF0000BFFB7D002B09D1A0
:104D6800964B5B6D23F038027B689B6F9349134326
:104D78004B6501E0FB7DBB757B681B6803F0020394
:104D8800002B38D07B685B6F052B21D801A252F825
:104D980023F000BFDF4D0008B54D0008C74D0008DF
:104DA800DF4D0008DF4D0008DF4D00087B68043345
:104DB8000121184600F0F6FA0346FB750CE07B6803
:104DC80024330121184600F09FFB0346FB7503E0DE
:104DD8000123FB7500E000BFFB7D002B09D1774B59
:104DE8005B6D23F007027B685B6F744913434B6567
:104DF80001E0FB7DBB757B681B6803F00403002B97
:104E08003AD07B68D3F89030052B21D801A252F80C
:104E180023F000BF5F4E0008354E0008474E0008DB
:104E28005F4E00085F4E00085F4E00087B68043341
:104E38000121184600F0B6FA0346FB750CE07B68C2
:104E480024330121184600F05FFB0346FB7503E09D
:104E58000123FB7500E000BFFB7D002B0AD1574BF7
:104E68009B6D23F007027B68D3F8903053491343B6
:104E78008B6501E0FB7DBB757B681B6803F0200335
:104E8800002B4BD07B68D3F88C30B3F1A04F2ED0D9
:104E9800B3F1A04F28D8B3F1804F2AD0B3F1804F97
:104EA80022D8B3F1405F26D0B3F1405F1CD8B3F1EC
:104EB800005F10D0B3F1005F16D8002B1DD0B3F1FE
:104EC800805F11D17B6804330021184600F06AFA2C
:104ED8000346FB7512E07B6824330221184600F074
:104EE80013FB0346FB7509E00123FB7506E000BFD1
:104EF80004E000BF02E000BF00E000BFFB7D002B24
:104F08000AD12E4B5B6D23F0E0427B68D3F88C30DE
:104F18002A4913434B6501E0FB7DBB757B681B6821
:104F280003F04003002B4DD07B68D3F89830B3F5DD
:104F3800A05F2ED0B3F5A05F28D8B3F5805F2AD044
:104F4800B3F5805F22D8B3F5406F26D0B3F5406F34
:104F58001CD8B3F5006F10D0B3F5006F16D8002B2E
:104F68001DD0B3F5806F11D17B680433002118463A
:104F780000F018FA0346FB7512E07B68243302211F
:104F8800184600F0C1FA0346FB7509E00123FB75DA
:104F980006E000BF04E000BF02E000BF00E000BF81
:104FA800FB7D002B0CD1054B9B6D23F4E0527B68F5
:104FB800D3F89830014913438B6503E00044025845
:104FC800FB7DBB757B681B6803F08003002B4BD00F
:104FD8007B68D3F89C30B3F5204F2ED0B3F5204F23
:104FE80028D8B3F5004F2AD0B3F5004F22D8B3F52F
:104FF800C04F26D0B3F5C04F1CD8B3F5804F10D0A2
:10500800B3F5804F16D8002B1DD0B3F5005F11D132
:105018007B6804330021184600F0C4F90346FB7589
:1050280012E07B6824330221184600F06DFA03462B
:10503800FB7509E00123FB7506E000BF04E000BF33
:1050480002E000BF00E000BFFB7D002B0AD19D4BB2
:105058009B6D23F460427B68D3F89C3099491343D5
:105068008B6501E0FB7DBB757B681B6803F008035B
:10507800002B1AD07B68D3F88030B3F5805F0AD153
:105088007B6824330221184600F03EFA0346002BC1
:1050980001D00123BB758B4B5B6D23F440527B68B9
:1050A800D3F88030874913434B657B681B6803F04E
:1050B8001003002B1AD07B68D3F89430B3F5807FA7
:1050C8000AD17B6824330221184600F01DFA0346F2
:1050D800002B01D00123BB757A4B9B6D23F44072E2
:1050E8007B68D3F89430774913438B657B681B68DA
:1050F80003F40023002B34D07B68D3F8A030B3F539
:10510800003F1DD0B3F5003F17D8002B03D0B3F5EF
:10511800803F09D011E07B6804330021184600F075
:1051280041F90346FB750CE07B68243302211846DD
:1051380000F0EAF90346FB7503E00123FB7500E084
:1051480000BFFB7D002B0AD15E4B9B6D23F44032E0
:105158007B68D3F8A0305B4913438B6501E0FB7D86
:10516800BB757B681B6803F48023002B33D07B68F6
:10517800D3F88430B3F5401F1CD0B3F5401F16D8C0
:10518800B3F5801F03D0B3F5001F07D00FE04D4BD8
:10519800DB6A4C4A43F40033D3620CE07B68243367
:1051A8000121184600F0B0F90346FB7503E001231E
:1051B800FB7500E000BFFB7D002B0AD1414B5B6D06
:1051C80023F440127B68D3F884303E4913434B657F
:1051D80001E0FB7DBB757B681B6803F48033002B03
:1051E80029D07B68DB6C002B03D0B3F5803F07D058
:1051F8000FE0344BDB6A334A43F40033D3620BE0ED
:105208007B6804330221184600F0CCF80346FB758E
:1052180002E00123FB7500BFFB7D002B09D1294B60
:10522800DB6C23F480327B68DB6C26491343CB6448
:1052380001E0FB7DBB757B681B6803F00053002B06
:105248000AD07B6824330221184600F05DF9034632
:10525800002B01D00123BB757B681B6803F4003366
:10526800002B33D07B68DB6FB3F5407F17D0B3F5E5
:10527800407F11D8B3F5007F13D0B3F5007F0BD86A
:10528800002B10D0B3F5807F06D10E4BDB6A0D4A98
:1052980043F40033D36207E00123FB7504E000BF49
:1052A80002E000BF00E000BFFB7D002B0CD1054BE6
:1052B8005B6D23F440727B68DB6F024913434B65D7
:1052C80004E000BF00440258FB7DBB757B681B6887
:1052D80003F48013002B08D0314B1B6D23F00042E0
:1052E8007B681B6F2E4913430B657B681B6803F0B3
:1052F8008053002B09D02A4B1B6923F480427B681A
:10530800D3F8B430264913430B617B681B6803F458
:105318000013002B08D0224B1B6D23F080727B6892
:105328009B6E1F4913430B657B681B6803F0804322
:10533800002B0DD01A4B1B69194A23F40043136143
:10534800174B1A697B68D3F8B830154913430B61BA
:105358007B681B68002B08DA114BDB6C23F040528A
:105368007B681B6D0E491343CB647B681B6803F491
:105378000003002B09D00A4B5B6D23F440027B68C5
:10538800D3F88830064913434B65BB7D002B01D108
:10539800002300E0012318461837BD4680BD00BF32
:1053A8000044025880B584B000AF786039600023AB
:1053B800FB73534B9B6A03F00303032B01D10123B7
:1053C80099E04F4B1B684E4A23F080631360FBF74C
:1053D8004BFFB86008E0FBF747FF0246BB68D31AEB
:1053E800022B01D9032386E0454B1B6803F00063B9
:1053F800002BF0D1424B9B6A23F47C327B681B68FC
:105408001B033F4913438B627B685B68013BC3F313
:1054180008027B689B68013B5B029BB21A437B686E
:10542800DB68013B1B0403F4FE031A437B681B691A
:10543800013B1B0603F0FE43314913438B63304B9A
:10544800DB6A23F0C0027B685B692D491343CB629A
:105458002B4BDB6A23F020027B689B6928491343A6
:10546800CB62274BDB6A264A23F01003D362244B16
:10547800DA6B244B13407A68D269D200204913436F
:10548800CB631F4BDB6A1E4A43F01003D3623B68B1
:10549800002B06D11A4BDB6A194A43F40023D36266
:1054A8000FE03B68012B06D1154BDB6A144A43F425
:1054B8008013D36205E0124BDB6A114A43F40013F0
:1054C800D3620F4B1B680E4A43F080631360FBF7EF
:1054D800CBFEB86008E0FBF7C7FE0246BB68D31AEC
:1054E800022B01D9032306E0054B1B6803F0006378
:1054F800002BF0D0FB7B18461037BD4680BD00BF9F
:10550800004402580700FFFF80B584B000AF786000
:1055180039600023FB73534B9B6A03F00303032B8F
:1055280001D1012399E04F4B1B684E4A23F0805369
:105538001360FBF799FEB86008E0FBF795FE02469A
:10554800BB68D31A022B01D9032386E0454B1B689D
:1055580003F00053002BF0D1424B9B6A23F07C727E
:105568007B681B681B053F4913438B627B685B683C
:10557800013BC3F308027B689B68013B5B029BB25B
:105588001A437B68DB68013B1B0403F4FE031A43E0
:105598007B681B69013B1B0603F0FE43314913433B
:1055A8000B64304BDB6A23F440627B685B692D49EE
:1055B8001343CB622B4BDB6A23F400727B689B6935
:1055C80028491343CB62274BDB6A264A23F48073AE
:1055D800D362244B5A6C244B13407A68D269D200A8
:1055E800204913434B641F4BDB6A1E4A43F4807304
:1055F800D3623B68002B06D11A4BDB6A194A43F485
:105608008003D3620FE03B68012B06D1154BDB6AA0
:10561800144A43F40003D36205E0124BDB6A114AD3
:1056280043F08073D3620F4B1B680E4A43F08053DC
:105638001360FBF719FEB86008E0FBF715FE024699
:10564800BB68D31A022B01D9032306E0054B1B685C
:1056580003F00053002BF0D0FB7B18461037BD46F3
:1056680080BD00BF004402580700FFFF70B50D4D14
:105678000D4C641BA4100026A64209D10B4D0C4CFE
:1056880000F02EF8641BA4100026A64205D170BDB8
:1056980055F8043B98470136EEE755F8043B984720
:1056A8000136F2E76C5700086C5700086C57000881
:1056B800705700080A44914200F1FF3300D1704747
:1056C80010B511F8014B03F8014F9142F9D110BD03
:1056D80002440346934200D1704703F8011BF9E7DF
:1056E800F8B500BFF8BC08BC9E467047F8B500BFC7
:0856F800F8BC08BC9E46704797
:105700000000000000000000000000000000000099
:105710000000000001000000020000000300000083
:105720000400000000000000050000000000000070
:105730000000000000000000060000000000000063
:105740000000000000000000070000000000000052
:105750000102030401020304060708090001020311
:0C57600004050607080C10141820304047
:04576C00BD02000872
:045770009902000892
:105774000090D0030090D00310000000010000004E
:0400000508001111CD
:00000001FF
